:100000000C9462000C947F000C947F000C947F0091
:100010000C947F000C947F000C947F000C94D90109
:100020000C947F000C947F000C947F000C947F0054
:100030000C947F000C947F000C947F000C947F0044
:100040000C94C5000C947F000C947F000C947F00EE
:100050000C947F000C947F000C947F000C947F0024
:100060000C947F000C947F00020000000024002705
:10007000002A0000000000250028002B00000000DE
:1000800000230026002900040404040404040402DC
:100090000202020202030303030303010204081025
:1000A00020408001020408102001020408102000F2
:1000B0000000070002010000030406000000000029
:1000C0000000000011241FBECFEFD8E0DEBFCDBF7F
:1000D00011E0A0E0B1E0E6EFFCE002C005900D9277
:1000E000A232B107D9F711E0A2E2B1E001C01D923E
:1000F000A034B107E1F70E944B040C9481000C94EA
:100100000000F8940C9479060895EF92FF920F93F3
:100110001F93CF93DF93C0E0D0E0FE01E05FFE4F7E
:100120006081718188EE93E00E9415067B01FE01DB
:10013000E050FF4F608171810027F7FC0095102F80
:1001400088E0A80197010E943502C801B7010E940A
:10015000070526E636E646EA5FE30E946B050E9445
:10016000D404882777FD8095982F0E940D0188E0A0
:100170000E94C2012296C031D10579F6DF91CF915C
:100180001F910F91FF90EF9008951F920F920FB65D
:100190000F9211242F933F938F939F93AF93BF930D
:1001A0008091260190912701A0912801B091290109
:1001B00030912A010196A11DB11D232F2D5F2D37EE
:1001C00020F02D570196A11DB11D20932A01809387
:1001D000260190932701A0932801B09329018091D3
:1001E000220190912301A0912401B0912501019653
:1001F000A11DB11D8093220190932301A09324019E
:10020000B0932501BF91AF919F918F913F912F9115
:100210000F900FBE0F901F9018959B01AC017FB7F8
:10022000F8948091220190912301A0912401B09132
:10023000250166B5A89B05C06F3F19F00196A11D69
:10024000B11D7FBFBA2FA92F982F8827860F911D28
:10025000A11DB11D62E0880F991FAA1FBB1F6A95DF
:10026000D1F7BC012DC0FFB7F89480912201909185
:100270002301A0912401B0912501E6B5A89B05C0FA
:10028000EF3F19F00196A11DB11DFFBFBA2FA92F95
:10029000982F88278E0F911DA11DB11DE2E0880FB8
:1002A000991FAA1FBB1FEA95D1F7861B970B885E83
:1002B0009340C8F2215030404040504068517C4F3C
:1002C000211531054105510571F60895789484B5DD
:1002D000826084BD84B5816084BD85B5826085BD42
:1002E00085B5816085BDEEE6F0E080818160808328
:1002F000E1E8F0E01082808182608083808181600B
:100300008083E0E8F0E0808181608083E1EBF0E0D1
:10031000808184608083E0EBF0E080818160808375
:10032000EAE7F0E08081846080838081826080835E
:100330008081816080838081806880831092C10089
:100340000895813041F0813018F08230D1F409C035
:1003500010926E00089580916F008D7F80936F00E2
:100360000895809170008D7F8093700081E080936C
:10037000B0008091B100887F84608093B1001092BA
:10038000B30008951F93182F80912001811711F059
:100390009FEF06C0E8E6F0E094918FEF8093200194
:1003A000892F0E94A101812F60E00E9480041F918B
:1003B00008951F920F920FB60F9211242F933F931F
:1003C0004F935F936F937F938F939F93AF93BF935D
:1003D000EF93FF938091390190913A01A0913B01F5
:1003E000B0913C010097A105B10551F1E0913D01AB
:1003F000F0913E01808190913F0189278083809117
:10040000390190913A01A0913B01B0913C0118163D
:1004100019061A061B06C4F48091390190913A011D
:10042000A0913B01B0913C010197A109B1098093D2
:10043000390190933A01A0933B01B0933C0104C071
:10044000809120010E94C201FF91EF91BF91AF9175
:100450009F918F917F916F915F914F913F912F91DC
:100460000F900FBE0F901F9018952F923F925F92A2
:100470006F927F928F929F92AF92BF92CF92DF92B4
:10048000EF92FF920F931F93DF93CF9300D000D092
:10049000CDB7DEB7A82F1B0129833A834B835C833A
:1004A000809120018A1721F4E8E6F0E0549082C0A0
:1004B0008F3F09F0DAC1A0932001E8E6F0E0549004
:1004C0002FEF521609F4D1C181E0581639F192E0AC
:1004D000591609F449C0552009F06CC014BC15BC6C
:1004E00084B5826084BD85B5816085BD2A2F30E0EA
:1004F000F901E957FF4FE491F0E0EE0FFF1FED58CF
:10050000FF4F859194919093300180932F01255650
:100510003F4FF9018491809331014EC010928000C9
:100520001092810080918100886080938100809189
:1005300081008160809381002A2F30E0F901E95722
:10054000FF4FE491F0E0EE0FFF1FED58FF4F859154
:100550009491909337018093360125563F4FF901CE
:1005600084918093380128C01092B0001092B1009D
:100570008091B00082608093B0008091B100816072
:100580008093B1002A2F30E0F901E957FF4FE49141
:10059000F0E0EE0FFF1FED58FF4F8591949190937F
:1005A0003E0180933D0125563F4FF9018491809390
:1005B0003F0102C057FC59C18A2F61E00E945A04D2
:1005C000552021F0F2E05F1609F0BEC03101882409
:1005D000992460E072E18AE790E0A40193010E940F
:1005E0004A0659016A01860175010894E108F1087B
:1005F000010911092FEFE216F1040105110509F0B7
:1006000008F499C060E472E48FE090E0A4019301E3
:100610000E944A0679018A010894E108F10801095B
:10062000110982E05816C1F49FEFE916F1040105A3
:10063000110509F008F484C060E970ED83E090E0F2
:10064000A40193010E944A0679018A010894E108F5
:10065000F1080109110983E0AFEFEA16F104010581
:10066000110509F008F468C068E478EE81E090E0D4
:10067000A40193010E944A0679018A010894E108C5
:10068000F10801091109552011F483E01DC0B2E001
:100690005B1611F084E018C0EFEFEE16F1040105CF
:1006A000110509F008F4DFC064E274EF80E090E027
:1006B000A40193010E944A0679018A010894E10885
:1006C000F1080109110985E0FFEFEF16F1040105BA
:1006D000110591F188F162E17AE780E090E0A401F0
:1006E00093010E944A0679018A010894E108F10801
:1006F00001091109552011F086E001C084E02FEFB7
:10070000E216F10401051105B9F0B0F0C601B5011A
:1007100020E034E040E050E00E944A0679018A017E
:100720000894E108F10801091109552011F087E04A
:1007300008C085E003C081E0552019F485BD3AC0AA
:1007400082E08093B10036C05101CC24DD2460E00A
:1007500072E18AE790E0A60195010E944A067901BC
:100760008A010894E108F1080109110980E0E816FE
:1007700080E0F80681E0080780E0180710F491E0B7
:1007800010C068E478EE81E090E0A60195010E9437
:100790004A0679018A010894E108F1080109110962
:1007A00093E0A1E05A1631F480918100887F982B64
:1007B0009093810089819A81AB81BC810097A105CA
:1007C000B10529F48FEF9FEFAFEFBFEF13C0220CFD
:1007D000331CB10180E090E029813A814B815C813A
:1007E0000E94F60528EE33E040E050E00E94280623
:1007F000C901DA01E1E05E16A1F0F2E05F1619F13D
:10080000552099F5E7BC80932B0190932C01A09380
:100810002D01B0932E0180916E00826080936E0056
:1008200024C0F0928900E092880080933201909376
:100830003301A0933401B093350180916F00826041
:1008400080936F0012C0E092B300809339019093BF
:100850003A01A0933B01B0933C018091700082600B
:100860008093700002C084E06CCF0F900F900F90C7
:100870000F90CF91DF911F910F91FF90EF90DF903C
:10088000CF90BF90AF909F908F907F906F905F9030
:100890003F902F900895CF93DF930E9466010E94AE
:1008A0008500C0E0D0E00E9484002097E1F30E9420
:1008B0000000F9CF482F50E0CA0185569F4FFC0138
:1008C000249149575F4FFA0184918823C1F0E82FA2
:1008D000F0E0EE0FFF1FE759FF4FA591B49166239B
:1008E00041F49FB7F8948C91209582238C939FBFFD
:1008F00008959FB7F8948C91822B8C939FBF089595
:10090000482F50E0CA0181559F4FFC012491CA0134
:1009100085569F4FFC01949149575F4FFA013491DE
:10092000332309F440C0222351F1233071F02430E5
:1009300028F42130A1F0223011F514C02630B1F096
:100940002730C1F02430D9F404C0809180008F7723
:1009500003C0809180008F7D8093800010C084B59B
:100960008F7702C084B58F7D84BD09C08091B000AF
:100970008F7703C08091B0008F7D8093B000E32F0C
:10098000F0E0EE0FFF1FED58FF4FA591B4912FB788
:10099000F894662321F48C919095892302C08C9160
:1009A000892B8C932FBF089504D06894B1118DC00A
:1009B000089570D088F09F5790F0B92F9927B751BC
:1009C000A0F0D1F0660F771F881F991F1AF0BA9513
:1009D000C9F712C0B13081F077D0B1E0089574C08A
:1009E000672F782F8827B85F39F0B93FCCF3869509
:1009F00077956795B395D9F73EF490958095709566
:100A000061957F4F8F4F9F4F0895E89409C097FBE2
:100A10003EF490958095709561957F4F8F4F9F4FD5
:100A20009923A9F0F92F96E9BB279395F695879519
:100A300077956795B795F111F8CFFAF4BB0F11F4DC
:100A400060FF1BC06F5F7F4F8F4F9F4F16C0882383
:100A500011F096E911C0772321F09EE8872F762FB9
:100A600005C0662371F096E8862F70E060E02AF0FA
:100A70009A95660F771F881FDAF7880F96958795E6
:100A800097F9089557FD9058440F551F59F05F3F4F
:100A900071F04795880F97FB991F61F09F3F79F0A0
:100AA00087950895121613061406551FF2CF469522
:100AB000F1DF08C0161617061806991FF1CF8695A4
:100AC0007105610508940895E894BB276627772788
:100AD000CB0197F908950BD078C069D028F06ED07B
:100AE00018F0952309F05AC05FC01124EECFCADF79
:100AF000A0F3959FD1F3950F50E0551F629FF00131
:100B0000729FBB27F00DB11D639FAA27F00DB11D89
:100B1000AA1F649F6627B00DA11D661F829F222712
:100B2000B00DA11D621F739FB00DA11D621F839F99
:100B3000A00D611D221F749F3327A00D611D231F6F
:100B4000849F600D211D822F762F6A2F11249F57BD
:100B500050408AF0E1F088234AF0EE0FFF1FBB1FE0
:100B6000661F771F881F91505040A9F79E3F51057F
:100B700070F014C0AACF5F3FECF3983EDCF386958B
:100B800077956795B795F795E7959F5FC1F7FE2B2A
:100B9000880F911D9695879597F9089597F99F6706
:100BA00080E870E060E008959FEF80EC08950024F5
:100BB0000A941616170618060906089500240A94C2
:100BC00012161306140605060895092E0394000C48
:100BD00011F4882352F0BB0F40F4BF2B11F460FFD7
:100BE00004C06F5F7F4F8F4F9F4F0895629FD0016A
:100BF000739FF001829FE00DF11D649FE00DF11DD8
:100C0000929FF00D839FF00D749FF00D659FF00D86
:100C10009927729FB00DE11DF91F639FB00DE11D73
:100C2000F91FBD01CF011124089597FB092E072656
:100C30000AD077FD04D049D006D000201AF4709570
:100C400061957F4F0895F6F7909581959F4F089590
:100C5000A1E21A2EAA1BBB1BFD010DC0AA1FBB1FC0
:100C6000EE1FFF1FA217B307E407F50720F0A21B32
:100C7000B30BE40BF50B661F771F881F991F1A949F
:100C800069F760957095809590959B01AC01BD01C9
:100C9000CF01089597FB092E05260ED057FD04D0ED
:100CA000D7DF0AD0001C38F4509540953095219537
:100CB0003F4F4F4F5F4F0895F6F790958095709591
:100CC00061957F4F8F4F9F4F0895AA1BBB1B51E12A
:100CD00007C0AA1FBB1FA617B70710F0A61BB70BAC
:100CE000881F991F5A95A9F780959095BC01CD0151
:060CF0000895F894FFCF07
:100CF6000601C400C400DC00C4000000F7000601C1
:100D060004000800080004000400040004000400B5
:020D1600FF00DC
:00000001FF
